:100000000C941E060C94F8270C9425280C94460694
:100010000C9446060C9446060C9446060C94460630
:100020000C9446060C9446060C94EF120C9446066B
:100030000C9446060C9446060C9446060C94460610
:100040000C9452280C9446060C94402C0C94832C4F
:100050000C9446060C9446060C9446060C944606F0
:100060000C9446060C9446067818DA18B918BC1891
:10007000BF18C218C518C818CB18DA18D4180C1A2B
:100080000E1A0E1A0C1A0E1A0E1A0E1A0E1A0E1A32
:100090000E1A0E1A0E1A0E1A0E1A0E1A0E1A0E1A20
:1000A00092190E1A0E1A0E1A0E1A0E1A03190E1A99
:1000B0000E1A0E1A0E1A0E1A0E1A0E1A0E1A0E1A00
:1000C0000E1A0E1A0E1A0E1A0E1A0E1A9E199E19D2
:1000D0009E199E199E199E199E199E199E190E1AF7
:1000E0000E1A0E1A0E1A0E1A0E1A03199D199D19C0
:1000F0009D199D190E1AAB19B119B719BD19C3195C
:10010000C919CF19D519DF19E919F319FD194419BE
:1001100006190E1A0E1A0E1A0E1A92190E1A0E1A25
:100120000E1A0E1A0E1A0E1A0E1A0E1A9C199C1975
:100130009C199C190E1AAB19B119B719BD19C3191D
:10014000C919CF19D519DF19E919F319FD1944197E
:1001500006190E1A0E1A0E1A0E1A9219411A411A7F
:10016000411A411A411A411A411A411A411A411AB7
:10017000411A411A411A581B581B581B581B581B2F
:10018000581B861A901A9A1AA41A021B0C1B1B1BC6
:100190002C1BB41CC91CD51CDE1CED1C121D1B1D08
:1001A000641D2D1D77207D2083208A209820BA2071
:1001B000D820456E746572206D656E752E2E2E00EA
:1001C000546F67676C6564206D6963726F50504D42
:1001D00000546F67676C656420696E76657274653C
:1001E000642050504D2100546F67676C6564205443
:1001F00058206D7574696E672100546F67676C6570
:10020000642074656C656D65747279210050726F3D
:10021000746F636F6C206572726F72207769746897
:100220002052580054696D656F7574207768656E4B
:1002300020636F6E6E656374696E6720746F205201
:100240005800507265737320616E79206B65792058
:10025000746F2063616E63656C00436F6E6E6563DF
:1002600074696E6720746F2052582C20706F776508
:100270007220757020746865205258202877697440
:10028000682062696E6420706C7567206966206EF4
:100290006F74207573696E6720616C776179732064
:1002A00062696E642900546F67676C656420276912
:1002B0006D6D656469617465206F75747075742700
:1002C00000546F67676C65642027736C61766520E6
:1002D0006D6F64652700546F67676C6564202761E4
:1002E0006C776179732062696E642700546F676769
:1002F0006C65642050504D206368616E6E656C20A3
:100300006C696D69740053657420525353492069B8
:100310006E6A656374696F6E206368616E6E656C8A
:100320002028303D3D64697361626C652900536526
:10033000742050504D206D696E696D756D20737914
:100340006E630053657420626561636F6E20696E31
:1003500074657276616C0053657420626561636FC9
:100360006E2064656C617900536574206265616319
:100370006F6E206672657175656E637920696E2097
:10038000487A3A20303D64697361626C652C205074
:10039000783D504D52206368616E6E656C20782CFC
:1003A0002046783D465253206368616E6E656C202E
:1003B00078005365742050574D2073746F7020641B
:1003C000656C61792028302064697361626C6564B2
:1003D0002C20312D323535203D3D20302E317320FB
:1003E0002D2035306D696E29005365742050504DB5
:1003F0002073746F702064656C61792028302064EC
:10040000697361626C65642C20312D323535203D75
:100410003D20302E3173202D2035306D696E29003E
:10042000536574206661696C736166652064656CF0
:1004300061792028302064697361626C65642C20C6
:10044000312D323535203D3D20302E3173202D2089
:1004500035306D696E29002A2A2A2A2A2A2A2A2A50
:100460002A2A2A2A2A2A2A2A2A2A2A2A2A2A2A2AEC
:100470002A2A2A2A0052582041636B6564202D20C5
:1004800072657665727420737563636573736675E0
:100490006C21002A2A2A2A2A2A2A2A2A2A2A2A2AAD
:1004A0002A2A2A2A2A2A2A2A2A2A2A2A2A2A2A2AAC
:1004B000002A2A2A2A2A2A2A2A2A2A2A2A2A2A2AC6
:1004C0002A2A2A2A2A2A2A2A2A2A2A2A2A2A00528E
:1004D000582041636B6564202D20757064617465DC
:1004E000207375636365737366756C21002A2A2A0D
:1004F0002A2A2A2A2A2A2A2A2A2A2A2A2A2A2A2A5C
:100500002A2A2A2A2A2A2A2A2A2A0056616C696457
:100510002063686F69636573206172653A205B319F
:100520005D2D5B31365D20286368616E6E656C20E1
:10053000312D31362900536574206F7574707574D0
:1005400020666F7220706F727420005B585D2061AE
:10055000626F7274206368616E67657320616E6498
:10056000206578697420525820636F6E6669670051
:100570005B535D20736176652073657474696E6783
:100580007320746F205258005B525D20726576654F
:1005900072742052582073657474696E6773207486
:1005A0006F2064656661756C747300557365206EA9
:1005B000756D62657273205B312D445D20746F2010
:1005C0006564697420706F727473205B452D515D92
:1005D00020666F722073657474696E677300202DD6
:1005E00020726563656976657220636F6E66696700
:1005F000757261746F722C20727820737720000AF4
:100600000A6F70656E4C52536E67200053657420FC
:1006100073657269616C2062617564726174653AB8
:10062000200056616C69642063686F696365733A82
:100630002031202D20342B34202F2032202D203823
:10064000202F2033202D20382B34202F2034202D14
:10065000203132202F2035202D2031322B34202FF5
:100660002036202D20313600536574204368616E9A
:100670006E656C20636F6E6669673A20005365741F
:100680002044617461726174652028302D32293AEA
:10069000200053657420486F70206368616E6E653A
:1006A0006C7320286D61782032342C207365706162
:1006B000726174656420627920636F6D6D61732966
:1006C0002076616C69642076616C75657320312DCC
:1006D0003235353A2000536574206368616E6E656B
:1006E0006C2073706163696E6720287831306B48C5
:1006F0007A293A200053657420524620706F77653E
:10070000722028302D37293A200053657420524634
:10071000206D6167696320286865782920652E67E8
:100720002E20307844454144463030443A2000532E
:1007300065742062617365206672657175656E63AC
:10074000792028696E20487A293A20005B5A5D207A
:10075000656E746572207265636569766572206383
:100760006F6E66696775726174696F6E2075746902
:100770006C79005B465D20646973706C61792061FF
:10078000637475616C206672657175656E63696509
:10079000732075736564005B525D2063616C6375E3
:1007A0006C6174652072616E646F6D206B65792079
:1007B000616E6420686F70206C697374005B495DC2
:1007C000207265696E697469616C697A6520736508
:1007D0007474696E677320746F20736B65746368DB
:1007E0002064656661756C7473005B585D2072658A
:1007F00076657274206368616E67657320616E64EC
:100800002065786974206D656E75005B535D20739B
:100810006176652073657474696E677320746F20E8
:10082000454550524F4D20616E64206578697420B3
:100830006D656E7500557365206E756D62657273BA
:10084000205B302D395D20746F20656469742070E1
:100850006172616D657465727300202D2053797328
:1008600074656D20636F6E66696775726174696F18
:100870006E000A0A6F70656E4C52536E672000510D
:1008800029204F7574707574206265666F726520DB
:100890006C696E6B20283D465329203A2000502970
:1008A00020536C617665206D6F64652028657870D3
:1008B0006572696D656E74616C293A20004F29205C
:1008C00054696D65642042494E44206174207374FC
:1008D000617274757020203A20004E292050504DCE
:1008E000206F7574707574206C696D69746564200F
:1008F000202020203A200044495341424C454400E6
:100900004D292050504D205253534920746F20637D
:1009100068616E6E656C202020203A20004C2920F2
:1009200050504D206D696E696D756D2073796E63E1
:10093000202875732920203A200044495341424C15
:100940004544004B29204661696C736166652062ED
:100950006561636F6E20696E74762E2028312D32AA
:10096000353573293A20004A29204661696C736144
:10097000666520626561636F6E2064656C617920D5
:1009800028302D323535203D3E20313073202D204A
:100990003135306D696E293A200049292046616958
:1009A0006C7361666520626561636F6E206672714B
:1009B0002E203A200048292050574D2073746F7024
:1009C0002064656C6179202020202020203A2000BE
:1009D00047292050504D2073746F702064656C61FE
:1009E00079202020202020203A200046292046611E
:1009F000696C736166652064656C617920202020D4
:100A00002020203A200050574D206368616E6E65AB
:100A10006C200066756E6374696F6E3A2000292041
:100A2000706F72742000506F776572546F776572C3
:100A300000445446205548462033322D62697420C4
:100A400031306368004F70656E4C52536E67525878
:100A5000206D696E6920342F36636800466C7974A6
:100A6000726F6E2F4F72616E6765525820554846FF
:100A70002038636800525820747970653A20004429
:100A8000697361626C656400487A00203D3D200016
:100A900043616C63756C61746564207061636B6540
:100AA0007420696E74657276616C3A200042292068
:100AB0004D6963726F202868616C66292050504D23
:100AC000202020203A00412920496E766572746505
:100AD000642050504D20696E20202020203A0030A4
:100AE00029204D7574652062757A7A657220286DAB
:100AF0006F73746C79293A003929205365726961E2
:100B00006C2062617564726174653A00736D617224
:100B100074506F7274004672536B79005472616E38
:100B200073706172656E740044697361626C6564B0
:100B30000038292054656C656D657472793A2020FF
:100B40002020202020003729204368616E6E656CCC
:100B500020636F6E6669673A202000362920446161
:100B60007461726174652028302D32293A2020206A
:100B700000352920486F70206368616E6E656C7364
:100B80003A2020202020003429204368616E6E65C1
:100B90006C2073706163696E673A202000332920EE
:100BA000524620706F7765722028302D37293A2001
:100BB0002020003229205246206D616769633A2067
:100BC0002020202020202020003129204261736530
:100BD000206672657175656E63793A202020000089
:100BE00000000700020100000304060000000000EE
:100BF00000000001020408102040800102040810D7
:100C00002001020408102004040404040404040263
:100C10000202020202030303030303000000002395
:100C2000002600290000000000250028002B0000FD
:100C3000000000240027002A0000712D11241FBE8F
:100C4000CFEFD8E0DEBFCDBF13E0A0E0B1E0E0EF32
:100C5000F0E602C005900D92A83CB107D9F716E066
:100C6000A8ECB3E001C01D92AE38B107E1F71CE07B
:100C7000CCE3DCE004C02297FE010E947A2ECA3346
:100C8000D107C9F70E94AD2D0C9476300C9400006A
:100C900080917305813019F482E08093730580910F
:100CA0007305833019F484E0809373050895A89543
:100CB0000895DC01ED91FC910190F081E02D099502
:100CC00008952091740530917505382748E0C901D1
:100CD000880F991F37FF06C09C0151E2252750E17C
:100CE000352701C09C01415091F730937505209341
:100CF0007405089588E38093760580E092ECA1E086
:100D0000B0E08093770590937805A0937905B09330
:100D10007A0587E08093830580EC9AECA9E8B6E336
:100D200080937B0590937C05A0937D05B0937E0511
:100D300085E0809384058DEE9EEFADEABEED809355
:100D40007F0590938005A0938105B0938205E5E827
:100D5000F5E080E090E0863028F4DC01AE54BC4F32
:100D60002C9101C020E0219301968831910599F7DB
:100D700082E080939D058AE080939E05089580EC33
:100D800097EFAAEBB7E38093BB059093BC05A093C4
:100D9000BD05B093BE0580E090E0A0E0B0E5809393
:100DA000BF059093C005A093C105B093C205E3ECC5
:100DB000F5E080E081938F5F8031E1F70895A0E056
:100DC000B0E0E5EEF6E00C94432ED82F0E94A82860
:100DD0006115710581059105C9F30E94E62E1092F7
:100DE0007F05109280051092810510928205C4E063
:100DF000812C912C54018A94C0907F05D09080055D
:100E0000E0908105F0908205FE2CED2CDC2CCC24AA
:100E10000E94E12EA50194010E94222E6C0D7D1DE1
:100E20008E1D9F1D60937F057093800580938105C3
:100E300090938205C15001F7DD2309F450C005E805
:100E400015E0E801A12CB12C62E3C62ED12CE12CD7
:100E5000F12C8881882309F442C0B39419F40E94CC
:100E60007A063DC00E94E12EA70196010E94222E23
:100E7000E1E0E60FA5E8B5E08A2F801B8A1520F493
:100E80008D918E13F9CFE9CF2091840530E0A0E158
:100E9000B7E20E94BA2D9B01AC01AE2FB0E00E94D8
:100EA000C92D40907B0550907C0560907D05709029
:100EB0007E05640D751D861D971D4090BB055090E5
:100EC000BC056090BD057090BE05461657066806C5
:100ED000790618F2E993A39488E1A812BACFCDB7A6
:100EE000DEB7E0E10C945F2E8436910520F4BC015E
:100EF00080E090E017C09C018E3B910528F42A55B4
:100F00003109AAE0B0E00CC0823D910528F4245BD1
:100F10003109A4E6B0E004C02D5C3109A8E5B2E0D7
:100F20000E94BA2DA4E6B0E09B01AC010E94C92D3D
:100F3000089590E08C599F4F0E947407089561E0D6
:100F40008AE00E94552960E08AE00E948E29089577
:100F5000892B11F061E001C060E08AE00E948E29D7
:100F6000089560E08CE00E94552961E08BE00E94CA
:100F7000552961E08DE00E94552960E082E00E94E1
:100F8000552961E084E00E945529089542E050E02F
:100F900068E476E080E00E94D8270895E3E0F0E07E
:100FA00089E080935700E491E67081E0E63009F033
:100FB00080E00895CF93DF93C82F0E94CE07882347
:100FC00081F0DFB781E080937205F8940E945706A4
:100FD00088E180936000C0936000C1110E945706B1
:100FE000DFBFDF91CF9108958F929F92AF92BF9212
:100FF000CF92DF92EF92FF92CF93FC01C0A5EC2F2E
:10100000E770F0E0E658FC4FA081B0E0C7FF03C0F6
:1010100024E130E002C02FE030E0FC0197A183E141
:10102000989FF0011124E25CFE4F80809180A280A5
:10103000B380A20FB31F20E43FE14DE750E00E94D0
:10104000D42DA50194010E94002E8C2F887149F4A3
:1010500069017A01E0EDCE0EE7E0DE1EE11CF11C35
:101060001BC0C7FF05C060E47AE88CE29EE004C0C4
:1010700060E07EEE8AEB9BE069017A01F8EBCF0E2F
:10108000FBE0DF1EE11CF11CA50194010E94002E73
:10109000C20ED31EE41EF51EC701B60169517C4F76
:1010A0008F4F9F4F28EE33E040E050E00E94002E2B
:1010B000A8EEB3E00E94C92DCF91FF90EF90DF9092
:1010C000CF90BF90AF909F908F9008958F3F9105E4
:1010D00051F048F0811522E0920738F081159340D5
:1010E00030F482E0089580E0089581E0089583E07F
:1010F0000895A0E0B0E0EFE7F8E00C944C2EEB018F
:101100008A01B82FB695A0E028813981F8012083A3
:101110002A813B8121832C813D8122832E813F8145
:101120002383688179814A815B812C813D81EE81B5
:10113000FF819F2F9295990F990F907C272F2370F5
:10114000922B252F2370220F220F922B232F2370F7
:101150002295207F922BF80194830B5F1F4F2896D6
:10116000AF5FBA1788F680FF24C0888199810E94FA
:101170006608D82E8A819B810E946608E82E8C81A1
:101180009D810E946608F82E8E819F810E946608CC
:10119000F0E4DF9EA001112490E1E99E900111246A
:1011A000242B282BE4E0FE9EB0011124262BF8010D
:1011B0002083CDB7DEB7E7E00C94682E803223E0C1
:1011C000920708F1883E23E0920740F48F51934044
:1011D000E4E096958795EA95E1F70895803D27E04C
:1011E000920718F48C5D93400895883928E092079F
:1011F00068F4885C974074E0969587957A95E1F756
:101200008D509C4F089580E090E008958FEF93E01B
:1012100008958C30910540F4A4E0880F991FAA9599
:10122000E1F7885D9C4F0895843F23E0920718F40E
:1012300084529C4F0895811524E0920740F486570C
:10124000934FF4E0880F991FFA95E1F7089580E92C
:1012500098E008959C013695279525753575821B74
:10126000930B9C0123733373969587959695879579
:1012700083739373820F931F9C0154E036952795D7
:101280005A95E1F7280F391F2F703F7041E051E068
:10129000249FC001259F900D349F900D1124892F0C
:1012A00008952D98882319F000002B9A02C00000A1
:1012B0002B9800002D9A000008952D9A000083B10C
:1012C0002D980000829581700895CF93DF93D82FD9
:1012D0005C9A2D985C98C8E08D2F80780E94510907
:1012E000DD0FC150C9F72D98DF91CF9108958F7709
:1012F0000E9465090895CF93DF93D82FC8E08D2F02
:1013000080780E945109DD0FC150C9F72D98DF91F7
:10131000CF910895CF93DF932D98C8E080E0D82F28
:10132000DD0F0E945D098D0FC150C9F7DF91CF918C
:1013300008950E9477090E948A095C9A0895A1E0A5
:10134000B0E0E5EAF9E00C94512E806869830E94D0
:1013500065096981862F0E947B095C9A2196E2E0EB
:101360000C946D2ECF93C0917F05C827E82FF0E035
:10137000EA58FA4F678589E70E949F096C2F8DE331
:101380000E949F096C2F82E40E949F09CF910895CB
:1013900086E20E9499090895CF93DF93EC016C8156
:1013A0008CE10E949F096D818DE10E949F096E81F1
:1013B0008EE10E949F096F8180E20E949F096885EB
:1013C00081E20E949F09698582E20E949F096A85E5
:1013D00083E20E949F096B8584E20E949F096C85CD
:1013E00085E20E949F096D858AE20E949F096E85B1
:1013F0008EE60E949F096F858FE60E949F0968898B
:1014000080E70E949F09698981E70E949F096A8994
:1014100082E70E949F09DF91CF910895CF92DF92DA
:10142000EF92FF92CF93DF936B017C01C11488E3AD
:10143000D8068CE9E8068CE1F80628F5C701B60164
:1014400020E836E948E950E00E94002EE90168975B
:1014500060E879E687E69FEF0E94DC2D6C0D7D1D2C
:101460008E1D9F1DF2E0660F771F881F991FFA954A
:10147000D1F721E732E040E050E00E94002EF22E4A
:10148000E32E80E421C0C701B60120E03DE241E344
:1014900051E00E94002EE901689760E073ED8EEC48
:1014A0009EEF0E94DC2D6C0D7D1D8E1D9F1D660F15
:1014B000771F881F991F21E732E040E050E00E942B
:1014C000002EF22EE32E80E66C2F6F71680F85E7F9
:1014D0000E949F096E2D86E70E949F096F2D87E766
:1014E0000E949F09DF91CF91FF90EF90DF90CF9006
:1014F0000895682F8DE60E949F0908958F929F920C
:10150000AF92BF92CF92DF92EF92FF92CF93DF9391
:10151000D82F83E00E9499098093710584E00E948E
:1015200099098093700560E086E00E949F0961E060
:1015300087E00E949F096FE789E00E949F0965E0AC
:101540008AE00E949F0962E18BE00E949F0965E1A9
:101550008CE00E949F096DEF8DE00E949F0960E082
:101560008EE00E949F09DD2319F08BE291E008C014
:1015700020919D0533E1239FC0011124825C9E4F81
:101580000E94CC096CE880E30E949F096FE082E32F
:101590000E949F0962E483E30E949F0980919E0557
:1015A00087FF02C064E101C06AE084E30E949F09F2
:1015B0006AE285E30E949F096DE286E30E949F092B
:1015C00064ED87E30E949F0960E088E30E949F0921
:1015D00060E089E30E949F09D11109C0C0907F0596
:1015E000D0908005E0908105F090820507C0C5E9A4
:1015F000CC2EC1ECDC2EED2CCEEDFC2ECAE38F2CD4
:101600009924AA24BB24682D8C2F0E949F09682D41
:1016100085E08C0F0E949F09FE2CED2CDC2CCC2445
:10162000CF5FCE3361F76FEF83E40E949F096FEFC6
:1016300084E40E949F096FEF85E40E949F096FEF89
:1016400086E40E949F09DD2311F066E002C06091EC
:1016500083058DE60E949F0960E089E70E949F094B
:10166000609184058AE70E949F0960E083E70E94F9
:101670009F0960E084E70E949F09D11109C0609131
:101680007B0570917C0580917D0590917E0504C05D
:1016900060EC7AEC89E896E30E940E0ADF91CF9124
:1016A000FF90EF90DF90CF90BF90AF909F908F9082
:1016B000089561E087E00E949F0964E28EE70E943E
:1016C0009F0963E088E00E949F0960E088E00E9433
:1016D0009F0965E087E00E949F0962E085E00E9423
:1016E0009F0983E00E9499098093710584E00E941C
:1016F000990980937005089583E00E949909809369
:10170000710584E00E9499098093700561E087E08B
:101710000E949F096AE070E080E090E00E94CB2880
:101720000E94590B00000895CF92DF92FF920F9311
:101730001F93CF93DF931F92CDB7DEB7082F162FDD
:101740008EE399830E949F09F02EC02E9981D92E95
:101750008C2D8F19811738F4F60161916F018FE795
:101760000E949F09F5CF64E085E00E949F0983E015
:101770000E9499098093710584E00E9499098093E1
:1017800070050E94A82860936C0570936D05809386
:101790006E0590936F0569E087E00E949F0981E0E4
:1017A000809373050F90DF91CF911F910F91FF9060
:1017B000DF90CF9008950F931F930E94940B809118
:1017C0007305813099F40E94A82800916C0510914E
:1017D0006D0520916E0530916F05601B710B820BBA
:1017E000930B603A76488140910548F380917305E8
:1017F000813031F46EE971E082EE95E00E94942A26
:101800001F910F9108950F931F938091730582305C
:1018100021F41092730581E020C08091730581301E
:10182000D9F40E94A82800916C0510916D052091B3
:101830006E0530916F05601B710B820B930B613A43
:1018400076488140910540F061E087E00E949F0961
:101850001092730582E001C080E01F910F910895FE
:10186000CF93DF93EC014AE050E06D2F70E082EE01
:1018700095E00E94622B6EE282EE95E00E94662A5D
:10188000BE0184E0769567958A95E1F76F707727BA
:101890004AE050E082EE95E00E94622B6EE282EE1A
:1018A00095E00E94662ABE016F7077274AE050E0FB
:1018B00082EE95E00E94622BDF91CF910895D82FA0
:1018C000C0E0CD1790F45E9A409A64E670E080E044
:1018D00090E00E94CB285E98409864E670E080E03B
:1018E00090E00E94CB28CF5FECCF6CE271E080E00B
:1018F00090E00E94CB28E4CF0F931F93CF93DF9308
:10190000EC01062F15E0115051F0CE010E945D3020
:10191000081741F0602FCE010E946530F4CF82E0BD
:101920000E945F0CDF91CF911F910F910895A0E06D
:10193000B0E0EDE9FCE00C94432E482E562EC0E0BA
:10194000D0E0612C712CE12CF12C00E010E0411072
:101950000CC06090D40586E4689E3001112459E1E2
:10196000E52EF12C0AEB15E01EC091E049120FC0E4
:101970006090D405E6E46E9E30011124FBE16F0E09
:10198000711C49E2E42EF12C06E715E00CC082E060
:10199000481209C028E1622E77247394EE24E39460
:1019A000F12C03ED15E043018C0E9D1E1092750580
:1019B000109274053401A62CA818B12CC30101960D
:1019C0006C01AE14BF04A8F4A00EB11E511006C0E5
:1019D000C3010E945D30F501808305C0F50160817F
:1019E000C3010E947C0CF50180810E9461063601D2
:1019F000E2CFC301511018C0C3010E945D30B82E60
:101A0000C6010E945D302B2D30E0322F2227282B7B
:101A100080917405909175058217930779F4C0E061
:101A2000D0E05524539493CF3601609175050E9400
:101A30007C0C60917405C6010E947C0CC05EDE4F78
:101A4000C13E92E0D90708F482CF852DCDB7DEB72D
:101A5000E0E10C945F2E61E082E00E94970C089513
:101A600060E082E00E94970C8091D305853020F0E1
:101A70001092D3050E942B0D8091D3058093D4053D
:101A8000089561E080E00E94970C61E081E00E948F
:101A9000970C089560E080E00E94970C882351F035
:101AA00060E081E00E94970C882321F08091760508
:101AB000883349F00E94BF060E947A0681E00E94A6
:101AC000DF060E94410D0895882319F06AEA71E04B
:101AD00002C06EEA71E082EE95E00E94942A0895B9
:101AE000FF920F931F93CF93DF9369EC7BE082EE1D
:101AF00095E00E94402A40917B0550917C056091C1
:101B00007D0570917E052AE030E082EE95E00E942E
:101B1000692B63EB7BE082EE95E00E94402A4091C6
:101B20007F0550918005609181057091820520E1CB
:101B300030E082EE95E00E94692B6DE97BE082EE59
:101B400095E00E94402A4AE050E06091830582EED1
:101B500095E00E94912B67E87BE082EE95E00E9481
:101B6000402A4AE050E06091840582EE95E00E94B0
:101B7000912B61E77BE082EE95E00E94402AC5E868
:101B8000D5E0F12C8E0188818823A9F0FF2031F067
:101B900061EB71E082EE95E00E94632A21964AE0B3
:101BA00050E0F801608182EE95E00E945A2BF39498
:101BB000F8E1FF12E7CF82EE95E00E946E2A6BE516
:101BC0007BE082EE95E00E94402A4AE050E060917E
:101BD0009D0582EE95E00E94912B66E47BE082EE0B
:101BE00095E00E94402AE0919E05E770F0E0EE0F3C
:101BF000FF1FEE57FC4F6081718182EE95E00E94DD
:101C0000942A61E37BE082EE95E00E94402A809175
:101C10009E058871883069F028F4811113C068E24C
:101C20007BE00CC0803141F0883161F46CE07BE0F6
:101C300005C06CE17BE002C066E17BE082EE95E0EE
:101C40000E94822A68EF7AE082EE95E00E94402AA4
:101C500040917705509178056091790570917A05EA
:101C60002AE030E082EE95E00E94692B6FED7AE089
:101C700082EE95E00E94402A8091BF0580710E940B
:101C8000640D66EC7AE082EE95E00E94402A809135
:101C9000BF0580740E94640D6DEA7AE082EE95E0E3
:101CA0000E94402A8091BF0580720E94640D60E905
:101CB0007AE082EE95E00E94402A86E795E00E9455
:101CC000F407AB01BC012AE030E082EE95E00E940F
:101CD0004B2B6BE87AE082EE95E00E94402A86E783
:101CE00095E00E94F4079B01AC0160E472E48FE090
:101CF00090E00E94002EBA01A9012AE030E082EEB5
:101D000095E00E944B2B68E87AE082EE95E00E9415
:101D1000822ACDB7DEB7E5E00C946A2E8F929F92AF
:101D2000AF92BF92CF92DF92EF92FF92811107C0E4
:101D30006FE77AE082EE95E00E94822A2FC090E061
:101D40000E94740724E630E040E050E00E94002E3C
:101D5000CA01B9012AE030E040E050E00E94002EC4
:101D600049015A016B017C012AE030E0B501A40170
:101D700082EE95E00E944B2B6EE282EE95E00E948F
:101D8000662A2AE030E0B701A60182EE95E00E94C3
:101D90004B2B63E782EE95E00E94A62AFF90EF901E
:101DA000DF90CF90BF90AF909F908F9008951F933A
:101DB000CF93DF9365E77AE082EE95E00E94402AB8
:101DC00080919F05813041F46CE57AE082EE95E0E8
:101DD0000E94822A10E050C0823019F465E47AE053
:101DE000F5CF843019F461E37AE0F0CF853091F7D4
:101DF00066E27AE0EBCFC12FD0E0C930D1050CF418
:101E000041C068E3610F82EE95E00E94662A6EE1B0
:101E10007AE082EE95E00E94402ABE016F5F7F4F1C
:101E20004AE050E082EE95E00E942A2B63E17AE0DE
:101E300082EE95E00E94402AC156DA4FE981E032F5
:101E400018F566E07AE082EE95E00E94402A8981EA
:101E5000803130F06DE673E082EE95E00E94632AF7
:101E600069816F7070E06F5F7F4F4AE050E082EEF3
:101E700095E00E94332B1F5F80914805181708F4E6
:101E8000BACF0FC061E3BECFEF70F0E0EE0FFF1FDF
:101E9000EE56FC4F6081718182EE95E00E94942A9B
:101EA000EACF6BEE79E082EE95E00E94402A8091C5
:101EB000B7050E948E0E60ED79E082EE95E00E94FB
:101EC000402A8091B8050E948E0E65EB79E082EE83
:101ED00095E00E94402A8091B9050E948E0E6AE921
:101EE00079E082EE95E00E94402A4091AF05509142
:101EF000B0056091B1057091B205411551056105BC
:101F0000710539F12AE030E082EE95E00E94692BFC
:101F100067E679E082EE95E00E94402A8091B30561
:101F20000E949907AB01BC012AE030E082EE95E007
:101F30000E94692B63E479E082EE95E00E94402ADA
:101F40004AE050E06091B40582EE95E00E94912B4A
:101F500006C06AE379E082EE95E00E94822A6DE194
:101F600079E082EE95E00E94402A6091B50570917B
:101F7000B6054AE050E082EE95E00E947B2B60E0DF
:101F800079E082EE95E00E94402A6091AE056034CF
:101F900050F470E06F5F7F4F4AE050E082EE95E0D2
:101FA0000E94332B06C067EF78E082EE95E00E9436
:101FB000822A6AED78E082EE95E00E94402A8091C4
:101FC000AD0580FF03C063EB71E002C067EB71E019
:101FD00082EE95E00E94942A6DEB78E082EE95E027
:101FE0000E94402A8091AD0582700E94640D6EE9C6
:101FF00078E082EE95E00E94402A8091AD058470E1
:102000000E94640D6FE778E082EE95E00E94402A1E
:102010008091AD0588700E94640DDF91CF911F9172
:1020200008950F931F93CF93DF93209145052F3F82
:10203000A9F56FEF75E082EE95E00E94402A84E8F2
:1020400093E00E94300C6EED75E082EE95E00E9408
:10205000402A80914605909147050E94300C6BEA1A
:1020600075E082EE95E00E94822A68E875E082EED3
:1020700095E00E94822A60E775E082EE95E00E947A
:10208000822A6BE475E082EE95E00E94822A82EE5D
:1020900095E00E946E2A0E94D70E68C012160CF0BE
:1020A00065C0332727FD30958091480590E0821761
:1020B00093070CF45BC066E375E082EE95E00E9446
:1020C000402A60914505772767FD70954AE050E00A
:1020D00082EE95E00E94332B6BE075E082EE95E096
:1020E0000E94402A10E008E2809149051817D0F5B7
:1020F000C12FD0E0CC0FDD1FC65BDA4F288130E066
:1021000080914505992787FD9095019728173907F4
:1021100039F56BEB71E082EE95E00E94632A4AE0AC
:1021200050E0602F82EE95E00E945A2B6FEB71E039
:1021300082EE95E00E94632AE981EF70F0E0EE0FF5
:10214000FF1FEE56FC4F6081718182EE95E00E9488
:10215000632A63EC71E082EE95E00E94632A0F5FD0
:102160001F5FC2CF82EE95E00E946E2ADF91CF9171
:102170001F910F910895FF920F931F93CF93DF93B9
:10218000C5E8D5E0F12C8E0188818823D1F165EC7A
:1021900071E082EE95E00E94632A4AE050E06F2DE4
:1021A00082EE95E00E945A2B62ED71E082EE95E09E
:1021B0000E94632A2196F801208130E0A0E1B7E275
:1021C0000E94BA2D9B01AC01A0918405B0E00E9451
:1021D000C92DAB01BC0180917B0590917C05A0913C
:1021E0007D05B0917E05480F591F6A1F7B1F2AE0AD
:1021F00030E082EE95E00E94692BF394F8E1FF1243
:10220000C2CFCDB7DEB7E5E00C946A2E1092DF04A2
:1022100085E6E0EEF4E0DF011D928A95E9F7089586
:10222000CF93C82F8F3719F0883009F045C0E0915F
:10223000DF04EE23D9F1E150E093DF04F0E0E05257
:10224000FB4F10826DE070E082EE95E00E9459062F
:10225000C0E08091DF04C81760F4EC2FF0E0E0529A
:10226000FB4F608170E082EE95E00E945906CF5FDF
:10227000F0CF60E270E082EE95E00E9459066DE0DA
:1022800070E082EE95E00E945906C0E08091DF0484
:10229000C81778F5EC2FF0E0E052FB4F608170E05A
:1022A00082EE95E00E945906CF5FF0CF67E082EEA4
:1022B00095E00E94662A1DC08B3119F40E94061118
:1022C0001AC08D30C1F08A30B1F08091DF048436BD
:1022D00068F76C2F70E082EE95E00E945906E0915D
:1022E000DF0481E08E0F8093DF04F0E0E052FB4FCB
:1022F000C08380E001C081E0CF910895CF93C82FC3
:102300000E94A8286093C8047093C9048093CA04EB
:102310009093CB04C093DD04CC2329F040E051EE30
:1023200060E070E004C040E855E260E070E082EEFA
:1023300095E00E94F02CCF9108959091CC04492F04
:102340004F7050E0BA016F5F7F4F292F30E0E4E01B
:1023500035952795EA95E1F76217730759F0FA0169
:10236000E353FB4F808381E0890F8F70907F892B2F
:102370008093CC0408956EE770E082EE95E00E94B1
:1023800059060895A3E1B1E0E8ECF1E10C94442E84
:10239000E5E8F5E0712C8191882321F0739428E120
:1023A0007212F9CF66ED71E082EE95E00E94942AF8
:1023B0004AE050E0672D82EE95E00E94912B80E08C
:1023C0000E947E0A0E94590B8E010E5F1F4FC12C86
:1023D000D12C7601C39466246A945C2C0E949C28BC
:1023E0004B015C012091840530E0A0E1B7E20E943E
:1023F000BA2D9B01AC01C701B6010E94DC2D2091D2
:102400007B0530917C0540917D0550917E05620FE2
:10241000731F841F951F2091BB053091BC0540910F
:10242000BD055091BE05261737074807590718F410
:10243000F801608229C08C2D0E94B20961E070E031
:1024400080E090E00E94CB28F80110820E949C2836
:10245000681979098A099B09643F714081059105D2
:1024600040F40E94C809F8019081981778F780839A
:10247000EDCF50FE05C05D9841985E9A409A04C029
:102480005D9A419A5E9840982FEFC21AD20AE20AEA
:10249000F20A0F5F1F4F8FEFC816D104E104F10459
:1024A00009F09BCFCE019395FC01D82E7FEF68EC0D
:1024B0002E2F281B271510F051E056C0DE01129672
:1024C00051E02FEF41E03D91321710F0322F01C063
:1024D000452F5F5F5F3F11F0232FF5CF4193242FEE
:1024E00030E0A1E0B0E0AC0FBD1FA20FB31F5C93C2
:1024F000413079F0DE01A20FB31F5C93423049F006
:10250000AFEFBFEFAC0FBD1FA20FB31F6C934E3FD9
:1025100078F6A2E0B0E0AC0FBD1FA20FB31F7C9312
:102520004D3F30F6A3E0B0E0AC0FBD1FA20FB31FCC
:102530006C93BECF452F242F30E0FC01E20FF31F38
:102540006081AFEFB0E0AC0FBD1FA20FB31F2C91A5
:10255000621748F44150DC01A40FB11D2C91208377
:102560006C934111E8CF5F5F571520F3372D3695F7
:1025700020E0231770F4DC01A20FB11D4C91522F03
:10258000530FFC01E50FF11D50815C9340832E5FDA
:10259000F0CFF5E8EF2EF5E0FF2E8C01802F8D199E
:1025A000871598F4F801C1908F014AE050E06C2D36
:1025B00082EE95E00E945A2B6CE282EE95E00E943A
:1025C000662AF701C1927F01E9CF82EE95E00E9471
:1025D0006E2A81E0CD5EDE4FEFE00C94602E1F92FC
:1025E0000F920FB60F9211241F932F933F934F9387
:1025F0005F936F937F938F939F93AF93BF93CF938B
:10260000DF93EF93FF93C0918600D0918700809174
:102610008704909188042091A904211155C09E013E
:10262000281B390B8091BF059091C005A091C10571
:10263000B091C20585FD02C036952795253C49E03D
:102640003407B8F140910A0150E060E070E02CE1FD
:10265000B695A795979587952A95D1F70097A105E7
:10266000B10521F481E090E0A0E0B0E08417950787
:10267000A607B707D8F480910A018F3FB9F040E070
:1026800080910A01481780F4842F90E0880F991FE9
:10269000FC01E757FB4F20813181FC01E55FFE4FD4
:1026A000318320834F5FECCF1092AA0410920A016D
:1026B0000BC02D3B82E0380720F080910A01803169
:1026C000D8F08FEF80930A01D0938804C0938704D9
:1026D000FF91EF91DF91CF91BF91AF919F918F913A
:1026E0007F916F915F914F913F912F911F910F902B
:1026F0000FBE0F901F90189510910A0181E0810F75
:1027000080930A01C9010E94DE08E12FF0E0EE0F7C
:10271000FF1FE757FB4F91838083D6CF83E08093E1
:1027200080008AE9809381008091BF0586FD05C005
:10273000809181008064809381008FEF9FEF909360
:1027400089008093880080916F00806280936F0081
:1027500008950E94300D8091D405843011F41092B8
:10276000D40508956F3018F086958058089589E053
:10277000689F802D11240895A0E0B0E0E2ECF3E121
:102780000C944B2EC82F0E94A82800913804109159
:10279000390420913A0430913B046B017C01C01A4A
:1027A000D10AE20AF30A9701860149E8C41643E117
:1027B000D406E104F10410F010923C046093380454
:1027C0007093390480933A0490933B042091A904B8
:1027D0008FEF820F8230D8F5E0913C04EE2309F4AC
:1027E0004EC1E13011F482E0B8C1E03108F034C1EB
:1027F00081E08E0F80933C04F0E0E757FB4FC083ED
:10280000803109F0ACC1EBE8F4E0213029F4A1817A
:10281000A695A695808108C080819181A92FA69553
:10282000A695A69596958795A03148F4B0E090E0DE
:10283000AA0FBB1FA55FBE4F11969C938E9310925B
:10284000AA04329684E0E939F807F9F688C1233002
:1028500009F005C1E0913C04E11104C0CF3009F05A
:102860007EC10DC1E83148F481E08E0F80933C04B5
:10287000F0E0E857FB4FC08372C1E83109F0ECC0CB
:10288000C111EAC040E050E0ABE0CA01B3E0880FFC
:10289000991FBA95E1F7A49F9001A59F300D1124CF
:1028A000F901E757FB4F6081E1817E2F77707595C5
:1028B0006795FC01EE0FFF1FE55FFE4F718360839C
:1028C000F901E657FB4FB081B695B695B695E18113
:1028D000FE2FF295FF0FF07E6F2F6B2BE695E6959E
:1028E000E6957E2F777075956795FC01EE0FFF1FBB
:1028F000E35FFE4F71836083F901E557FB4FB081C1
:10290000B295B695B695B370C181DC2FDD0FDD0FA2
:102910006D2F6B2BC295C695C695C370E281E17091
:10292000EE0FEE0F7E2F7C2B75956795FC01EE0F59
:10293000FF1FE15FFE4F71836083F901E357FB4F97
:10294000B081B695E181FE2FF795FF27F7956F2FA0
:102950006B2BE6957E2F777075956795FC01EE0FD2
:10296000FF1FEF5EFE4F71836083F901E257FB4F5B
:10297000B081B295BF70E181FE2FF295F07F6F2F8D
:102980006B2BE295EF707E2F777075956795FC0144
:10299000EE0FFF1FED5EFE4F71836083F901E1577B
:1029A000FB4FB081BB1FBB27BB1FC181DC2FDD0FDD
:1029B0006D2F6B2BCC1FCC27CC1FE281E370EE0F69
:1029C0007E2F7C2B75956795FC01EE0FFF1FEB5E4C
:1029D000FE4F71836083F901EF56FB4FB081B695CE
:1029E000B695E181FE2FF295FF0FFF0FF07C6F2F60
:1029F0006B2BE695E6957E2F777075956795FC01B4
:102A0000EE0FFF1FE95EFE4F71836083F901EE5602
:102A1000FB4F20812295269527703181E32FEE0F01
:102A2000EE0FEE0F6E2F622B732F729576957770E7
:102A300075956795FC01EE0FFF1FE75EFE4F7183F2
:102A400060834F5F5F4F4230510509F01ECF809188
:102A50009F0483FF1092AA0410923C0480C024308B
:102A600009F07DC060913C0461110BC0C83AB1F41B
:102A7000109275051092740588EA0E94610681E043
:102A80006CC0613019F4C093370404C0623031F473
:102A9000C09336048C2F0E9461065AC0E091360420
:102AA0002E2F30E0220F331F462F50E0C90102962F
:102AB000841795073CF0633268F7FA01EA57FB4F39
:102AC000C083E8CF2D5F3F4F8C2F90E0609174055D
:102AD000709175054217530749F4982F8827862768
:102AE0009727909375058093740532C0681779070E
:102AF00069F580913704813049F5E13118F080E1C2
:102B000080933604F0903604CAE8D4E000E010E088
:102B10000F15D0F4FE013197808190E0982F88271F
:102B20002881822B63E0969587956A95E1F70E944C
:102B3000DE08F801EE0FFF1FE55FFE4F91838083F3
:102B40000F5F1F4F2296E4CF1092AA0410923C040C
:102B500080913C04882319F08F5F80933C04CDB7AB
:102B6000DEB7E8E00C94672EE82FF0E0E654FA4F69
:102B7000E185E03150F4F894F0E0EE0FFF1FE55FDF
:102B8000FE4F80819181789408958EE08E0F8B3076
:102B900058F4F0E0E25FF10924E62E9FC0012F9F78
:102BA000900D11240C960895E03FF1F028F4E031E7
:102BB00061F0E13161F006C0ED3F81F0EE3F89F058
:102BC000E13F49F080E092E0089582E101C083E1B5
:102BD0000E94EA29089586E090E008958AEF93E044
:102BE00008958FEF93E0089580E090E00895A2E2C9
:102BF000B0E0EDEFF5E10C94412E9E012F5F3F4FC9
:102C000080E1D9011D928A95E9F764E072E082EED5
:102C100095E029A33AA30E94942A0E947C0B1D8A66
:102C20001E8A1F8A188E312C212C00E0812C912CB9
:102C3000540170EC472E7DE9572E78E5672E75E339
:102C4000772EE0E5CE2EE3ECDE2EE12CF12C84EFA6
:102C500091E0A0E0B0E08D8F9E8FAF8FB8A380ECA5
:102C600097EFAAEBB7E3898F9A8FAB8FBC8F80EC7D
:102C70009DE9A8E5B5E3898B9A8BAB8BBC8B82EE83
:102C800095E00E94A82B892B09F4E1C082EE95E023
:102C90000E94D52B9C0133272C32310509F442C008
:102CA000ACF42332310509F0ABC019821A821B82C1
:102CB0001C821D821E821F82188619861A861B8618
:102CC0001C861D861E861F86188A60C02434310526
:102CD00029F02335310509F4B2C092C064E482EED4
:102CE00095E00E94662A2AE030E040EC5DE968E564
:102CF00075E382EE95E00E94F42A6CE282EE95E0A4
:102D00000E94662A2AE030E040EC57EF6AEB77E356
:102D100082EE95E00E94F42A6CE282EE95E00E9439
:102D2000A62AADCF0F5F043009F0A9CF29813A81DF
:102D30004B815C81A8EEB3E00E94C92D698B7A8B30
:102D40008B8B9C8B2D813E814F8158850E94C92D94
:102D5000698F7A8F8B8F9C8F29853A854B855C850F
:102D60002D8F3E8F4F8F58A32D853E854F855889D7
:102D70000E94C92D6B017C0160323EE4730781051E
:102D8000910530F462E38CE10E949F0900E077CF67
:102D9000603345E774078105910510F462E2F3CFD3
:102DA00060345CE975078105910510F466E2EBCFAC
:102DB00080E5C81683ECD806E104F10410F462E162
:102DC000E2CF90E6C9169AEED906E104F10410F4B8
:102DD00065E1D9CFA0E7CA16A1E1DA06A1E0EA06CB
:102DE000F10410F461E0CFCFB0EACB16B6E8DB0611
:102DF000B1E0EB06F10410F463E0C5CF65E0C3CFAA
:102E000010ED180F1A3008F03ACFE1E0F0E0EC0FC7
:102E1000FD1F24E0029FE00DF11D1124208131816E
:102E200042815381AAE0B0E00E94C92D610F711D5B
:102E3000811D911D608371838283938320CF498894
:102E40005A886B887C88812C912C540118CF81146E
:102E50009104A104B10489F4C301B2010E940E0AD5
:102E600061E070E080E090E00E94CB281D8A1E8A1D
:102E70001F8A188E312C22242A948D8D9E8DAF8D21
:102E8000B8A188169906AA06BB06D0F40E94C80904
:102E90002D893E894F89588D280F311D411D511DA7
:102EA0002D8B3E8B4F8B588F381608F4382E821599
:102EB00008F4282E3FEF831A930AA30AB30A56C0D8
:102EC000C301B20128EE33E040E050E00E94002E42
:102ED000BA01A9012AE030E082EE95E00E944B2B76
:102EE0006CE282EE95E00E94662A4AE050E0632D93
:102EF00082EE95E00E945A2B6CE282EE95E00E94F1
:102F0000662A6D897E898F89988DA50194010E941A
:102F1000002EBA01A9012AE030E082EE95E00E947D
:102F20004B2B6CE282EE95E00E94662A4AE050E06C
:102F3000622D82EE95E00E945A2B6CE282EE95E0C3
:102F40000E94A62A4C0C5D1C6E1C7F1C898D9A8DDC
:102F5000AB8DBC8D84159505A605B70520F4498871
:102F60005A886B887C88812C912C540129893A8954
:102F70004B895C89283E33404105510509F07FCEDD
:102F8000A296E2E10C945D2EACE1B0E0EAECF7E150
:102F90000C944B2E0E94A8286B017C0181E00E94BA
:102FA0007E0A14E703E0198361E0CE0101960E94D6
:102FB000DB0B009373050E94590B6AEF70E080E011
:102FC00090E00E94CB2880917305833089F482EED3
:102FD00095E00E94A82B892B59F40E94A8286C190F
:102FE0007D098E099F096038734C894C9140D8F255
:102FF00080917305833009F44FC08FE70E947709F1
:103000000E948A098983843511F083E05CC00E94A4
:103010008A0910924605809347050E948A092091EB
:10302000460530914705280F311D30934705209301
:1030300046050E948A09809348050E948A09809368
:103040004905813110F7F12C0F2D10E080914905D1
:1030500090E0880F991F0817190740F40E948A0909
:10306000F801E65BFA4F8083F394EECF80E7898323
:1030700061E0CE0101960E94DB0B83E08093730533
:103080000E94590B62E370E080E090E00E94CB2840
:1030900080917305833011F482E015C08FE70E94A0
:1030A00077090E948A098983803509F0AECF0FE93C
:1030B00015E00E948A09F80181938F01F5E00A3B2F
:1030C0001F07B9F781E06C96E8E00C94672E8091B9
:1030D0004505992787FD9095A92FB92FFC013196B9
:1030E000EB30F10508F066C0EC5CFF4F0C94782ED5
:1030F00062E778E082EE95E00E94822A84E893E01D
:103100000E94300C6AE578E082EE95E00E94822A07
:1031100065E378E082EE95E00E94822A6BE078E039
:1031200082EE95E00E94822A6AEE77E082EE95E0D8
:103130000E94822A6DEB77E082EE95E00E94822A5F
:1031400067E977E082EE95E00E94822A63E777E004
:1031500082EE95E00E94822A6CE477E082EE95E0B0
:103160000E94822A82EE95E00E946E2A0E94700DD3
:1031700021C06FE277E01AC06AE077E017C065EF20
:1031800076E014C066ED76E011C062E976E00EC02C
:103190006DE776E00BC068E676E082EE95E00E948F
:1031A000822A62E276E002C06CE076E082EE95E090
:1031B0000E94822A6AE070E080E090E00E94CB28C2
:1031C00082EE95E00E94A82B892B29F082EE95E0F3
:1031D0000E94D52BF5CF0895ACE1B0E0E2EFF8E125
:1031E0000C944B2E909145059F3F09F023C1482F29
:1031F00050E0FA013A97EF36F10508F00FC1E15CB3
:10320000FF4F0C94782E61E172E0A0C06DE172E096
:1032100082EE95E00E94942A85E789838BE1EFE9AD
:10322000F5E0DE01129601900D928A95E1F76CE1CE
:10323000CE0101960E94DB0B0E94590B83E0809324
:10324000730568EC70E080E090E00E94CB288091EC
:103250007305843009F0E2C08FE70E9477090E946D
:103260008A098983853509F0D9C06DEE74E082EE54
:1032700095E00E94822A6FEC74E082EE95E00E9455
:10328000822A61EB74E096C065E372E082EE95E01D
:103290000E94942A89E6898361E0CE0101960E940A
:1032A000DB0B0E94590B83E08093730568EC70E0A0
:1032B00080E090E00E94CB2880917305843009F073
:1032C000ADC08FE70E9477090E948A0989838E0129
:1032D0000E5F1F4F7E014DE1E40EF11C0E948A0932
:1032E000F80181938F01EE15FF05C1F78BE1FE0117
:1032F0003296AFE9B5E001900D928A95E1F78981A8
:10330000893409F08BC063E974E082EE95E00E9495
:10331000822A65E774E082EE95E00E94822A67E5E2
:1033200074E048C06FE472E082EE95E00E94942A57
:103330008EEF8093450572C08052875080539091E4
:103340004805981708F066C06EE572E082EE95E0D9
:103350000E94942A63C084E18093450560E274E092
:1033600029C085E18093450569EE73E023C086E1BD
:103370008093450562EB73E01DC087E180934505AE
:1033800068E673E017C088E18093450567E573E060
:1033900011C089E18093450563E473E00BC08AE1C5
:1033A000809345056EE273E005C08BE1809345058F
:1033B00066E073E082EE95E00E94822A2FC06CEEF8
:1033C00072E082EE95E00E94822A8091AD0591E044
:1033D0001DC066ED72E082EE95E00E94822A809127
:1033E000AD0592E013C061EC72E082EE95E00E94C0
:1033F000822A8091AD0594E009C066EA72E082EE0F
:1034000095E00E94822A8091AD0598E089278093FB
:10341000AD058FEF809345050E94111082EE95E077
:103420000E94A82B892B09F45BC182EE95E00E94D3
:10343000D52BF4CF0E941011882309F451C180913B
:10344000DF04811104C08FEF8093450541C140E046
:1034500050E060E070E080EE94E00E94EF2E40913A
:103460004505042F112707FD1095212F312FF80155
:103470003197EB31F10508F01BC1E255FF4F0C9479
:10348000782E552747FD50952091480530E02417A8
:1034900035070CF40DC18B019C0101501109210964
:1034A0003109003211052105310558F0C090490558
:1034B000EBE4F5E0F12CD12CA8E2EA2E41505109C1
:1034C0000FC0FA01E156FA4F61506083D9C0DF01A5
:1034D00011972C9130E02417350729F0F394329698
:1034E000FC10F5CFCBC00E2D10E020E030E0061729
:1034F00017072807390741F42081DA01A156BA4F8E
:1035000011962C93DD24D394E394E8CF6F3F71059B
:103510008105910511F008F0CBC06093B705B0C0EC
:103520006F3F71058105910511F008F0C1C06093EE
:10353000B805A6C06F3F71058105910511F008F02F
:10354000B7C06093B9059CC02091E0042062203789
:10355000E9F440E050E060E070E081EE94E00E9429
:10356000EF2E9B01AC01DC01CB010197A109B10950
:103570000897A105B10508F0AEC0A4EDB0E30E9424
:10358000C92D6A5E7C4A8A46954E24C02636E9F4E7
:1035900040E050E060E070E081EE94E00E94EF2EA9
:1035A0009B01AC01DC01CB010197A109B10907978F
:1035B000A105B10508F08FC0A8EAB1E60E94C92DA7
:1035C000645E7C438E46944E05C06115710581058D
:1035D000910579F08B019C01005C1D49284535431C
:1035E0000130FAE51F07F2E62F07F2E03F0708F087
:1035F0005FC06093AF057093B0058093B105909361
:10360000B2053EC06F3F71058105910511F008F0CC
:103610004FC06093B30534C08B019C010150110968
:10362000210931090F3F11052105310508F040C07E
:103630006093B40525C08B019C01045C19402109ED
:1036400031090D344DE114072105310528F470933B
:10365000B6056093B50514C0611571058105910526
:1036600021F48FEF8093AE050BC0613471058105A5
:103670009105F0F461506093AE0502C0DD20C1F009
:103680008091DE0481111AC080917F0590918005A0
:10369000A0918105B09182050196A11DB11D809375
:1036A0007F0590938005A0938105B093820506C0A5
:1036B00060E772E082EE95E00E94942A0E94061173
:1036C0008FEF809345056AE082EE95E00E94A62A7E
:1036D0000E94111005C061E070E080E090E07ACFB8
:1036E0006C96E8E00C94672E6AE572E082EE95E055
:1036F0000E94822A62E472E082EE95E00E94822AB1
:1037000082EE95E00E94A82B892B31F082EE95E0A5
:103710000E94D52B0E94EC180E94C417823029F019
:10372000833051F46DE072E002C064E272E082EE38
:1037300095E00E94822A08958FEF809345051092AC
:10374000DE040E941110809145058E3F69F082EEE3
:1037500095E00E94A82B892BB1F382EE95E00E94A0
:10376000D52B0E94EC18EFCF08950F931F93109163
:1037700045051F3F09F0D2C0893409F457C000F550
:10378000883309F469C058F4803309F477C008F02D
:1037900061C08B3109F440C08132B1F1B9C08134CC
:1037A00009F487C030F4893309F466C0803461F1CC
:1037B000AFC0823409F48EC0863409F448C0A8C072
:1037C000823609F487C078F4883531F128F48235DF
:1037D000C1F18335E1F09CC08A3509F494C081368B
:1037E00009F467C095C0823761F128F4863679F113
:1037F0008936E1F08DC0883779F08A3709F483C0C3
:10380000833709F085C003C061E172E015C00E94F2
:10381000410D6EE872E004C00E944A0D68EA72E051
:1038200082EE95E00E94942A8EEF70C00E947A0684
:103830000E94BF0667EC72E082EE95E00E94942A37
:1038400067C081E00E94DF0660EE72E0F5CF0E9463
:10385000BB105EC080535AC06AEF71E082EE95E003
:103860000E94822A90919E0588E0890F8871977E38
:10387000892B80939E051AC089E048C067EE71E0ED
:1038800082EE95E00E94822A8091BF059091C0054A
:10389000A091C105B091C20520E182278093BF05A8
:1038A0009093C005A093C105B093C2051093450540
:1038B0002FC061ED71E082EE95E00E94822A809136
:1038C000BF059091C005A091C105B091C20540E42B
:1038D000842710C060EC71E082EE95E00E94822A9D
:1038E0008091BF059091C005A091C105B091C2051E
:1038F00020E282278093BF059093C005A093C10565
:10390000B093C20502C00E94741B8FEF80934505DF
:10391000809145058E3F09F0D4C0DDC00E94101192
:10392000882309F4D8C08091DF04811104C08FEF8F
:1039300080934505C6C040E050E060E070E080EE56
:1039400094E00E94EF2E00914505112707FD109588
:10395000212F312FF8013197E930F10508F0B4C07B
:10396000E753FF4F0C94782E8B019C01015C1D499D
:10397000284535430F3F19452246324008F0A4C080
:1039800060937B0570937C0580937D0590937E0505
:1039900077C060937F057093800580938105909335
:1039A000820581E08093DE046BC06830710581057B
:1039B000910508F089C06093830562C08B019C016A
:1039C00001501109210931090A301105210531057C
:1039D00008F07AC06093840553C061EB71E080EE1B
:1039E00094E00E94293010E0009799F00E94033083
:1039F000009779F0183130F4E12FF0E0EA58FA4FEF
:103A000087871F5F61EB71E080E090E00E942930C2
:103A1000EBCF1831A8F5E12FF0E0EA58FA4F1786FE
:103A20001F5FF7CF653071058105910508F04CC027
:103A300060939D0525C08B019C010150110921094E
:103A400031090630110521053105F0F520919E055B
:103A5000287F262B20939E0513C08B019C010150CB
:103A60001109210931090115124C2140310560F578
:103A700060937705709378058093790590937A0524
:103A80008091DE04811113C080917F0590918005A3
:103A9000A0918105B09182050196A11DB11D809371
:103AA0007F0590938005A0938105B09382050E94C5
:103AB00006118FEF809345056AE082EE95E00E9443
:103AC000A62A0E94671807C060E772E082EE95E0C0
:103AD0000E94942AECCF1F910F9108958FEF80934D
:103AE00045051092DE040E946718809145058E3FBF
:103AF00069F082EE95E00E94A82B892BB1F382EE4B
:103B000095E00E94D52B0E94B51BEFCF6AE070E0D4
:103B100080E090E00E94CB2882EE95E00E94A82BE6
:103B2000892B29F082EE95E00E94D52BF5CF0895E0
:103B3000CF93C82F682F82EE95E00E94022C9091BF
:103B40006A059C2790936A05CF910895A1E0B0E0A3
:103B5000ECEAFDE10C94512E99830E94981D998105
:103B6000892F0E94981D2196E2E00C946D2E1F93E0
:103B7000CF93DF93182FEB0110926A0565EB70E08D
:103B800082EE95E00E94590662E670E082EE95E0D2
:103B90000E945906812F0E94981DCE010E94A61DE9
:103BA000DF91CF911F91089560916A0582EE95E0B3
:103BB0000E94022C0895A1E2B0E0E1EEFDE10C9438
:103BC0004D2E7B018A018C3009F453C108F040C0AE
:103BD000863009F4BCC018F5833009F491C070F444
:103BE000813009F472C0823009F048C26BE170E0A4
:103BF00082E00E94B71D0FE915E078C0843009F417
:103C000087C0853009F03AC26091490570E0660FBF
:103C1000771F85E00E94B71D0AE415E086C0893051
:103C200009F4A7C070F4873009F49BC0883009F00C
:103C300025C261E070E088E00E94B71D8091D40544
:103C400023C28A3009F4CAC08B3009F4F2C016C20C
:103C50008A3609F475C1D8F4873609F43AC138F4C4
:103C6000853609F40EC1863609F41FC107C28836AD
:103C700009F437C1893609F001C261E070E089E6D4
:103C80000E94B71D0E947A060E94BF06F5C18D36BC
:103C900009F4D4C138F48B3609F491C18C3609F497
:103CA0009AC1ECC18E3609F4DCC1873C09F0E6C14B
:103CB00061E070E087EC0E94B71D81E00E94981DD2
:103CC0000E94D41D10926B05E3C169E270E081E0AF
:103CD0000E94B71D06E715E0F80181918F010E944F
:103CE000981DF5E00F391F07B9F7D0C1F801819190
:103CF0008F010E94981DF5E00A3B1F07B9F7C6C166
:103D000061E070E083E00E94B71D0E94C417BCC14F
:103D100061E070E084E00E94B71D81E00E94981D80
:103D20000E94D41D0E94F715B3C18091490590E00F
:103D3000880F991F98012A5435402817390708F031
:103D4000A5C1F80181918F010E94981DEECF62E01C
:103D500070E086E00E94B71D84E893E00E94A61DF3
:103D600095C161E070E087E00E94B71D8091480531
:103D70008BC186E6898361E0CE0101960E94DB0B50
:103D80000E94590B83E08093730568EC70E080E03B
:103D900090E00E94CB28809173058430D9F48FE79E
:103DA0000E9477090E948A098983863469F460E257
:103DB00070E089E00E94B71D10E20E948A090E940B
:103DC000981D1150D1F762C161E070E089E00E9456
:103DD000B71D52C161E070E089E053C169E170E054
:103DE0008AE00E94B71D82E08093BA052091720597
:103DF0008091BF059091C005A091C105B091C20509
:103E0000222311F0806801C08F778093BF059093C3
:103E1000C005A093C105B093C2050AEB15E0F801F7
:103E200081918F010E94981DF5E0033D1F07B9F7AE
:103E30002DC161E270E08BE00E94B71D8091AA0461
:103E40008F3F39F08091AA0491E0980F9093AA04D3
:103E500002C08091AA040E94981D10E0812F0E9448
:103E6000B4150E9409090E94A61D1F5F1031B1F709
:103E70000DC161E070E08CE00E94B71D8091D30518
:103E800003C161E070E085E60E94B71D89E2E81693
:103E9000F10409F0F8C0D801E6E7F5E08D918193CF
:103EA00085E0EF39F807D1F7E7C061E070E086E61A
:103EB0000E94B71DEBE1EE16F10409F0E4C0D80151
:103EC000EFE9F5E08D91819385E0EA3BF807D1F7C2
:103ED000D3C061E070E087E60E94B71D0E94410DEB
:103EE000CBC061E070E088E60E94B71D85E789835A
:103EF0008BE1EFE9F5E0DE01129601900D928A95D3
:103F0000E1F76CE1CE0101960E94DB0B0E94590B98
:103F100083E08093730560E273E080E090E00E94AC
:103F2000CB2880917305843009F0ADC08FE70E94E3
:103F300077090E948A098983853509F0A4C09CC04D
:103F400061E070E08AE60E94B71D89E6898361E03E
:103F5000CE0101960E94DB0B0E94590B83E08093F7
:103F6000730560E273E080E090E00E94CB288091CE
:103F70007305843009F087C08FE70E9477090E949B
:103F80008A0989838E010E5F1F4F7E01EDE1EE0EDF
:103F9000F11C0E948A09F80181938F01EE15FF053B
:103FA000C1F78BE1FE013296AFE9B5E001900D92C9
:103FB0008A95E1F78981893409F065C05DC061E0C7
:103FC00070E08BE60E94B71DF80180818093D405D4
:103FD0000E944A0D51C061E070E08CE60E94B71D5E
:103FE000F0E2EF16F10461F487E6898380E2F801DC
:103FF000DE01129601900D928A95E1F761E203C00D
:1040000087E4898361E0CE0101960E94DB0B0E9468
:10401000590B83E0809373056CE474E080E090E0DA
:104020000E94CB2880917305843069F58FE70E9448
:1040300077090E948A09873431F51EC061E070E07B
:104040008DE60E94B71D89E1E816F104E1F4D8017C
:10405000EAEBF5E08D91819385E0E33DF807D1F738
:104060000BC061E070E08EE60E94B71DF801808110
:104070008093D3050E942B0D81E006C061E070E0C3
:104080008AEC0E94B71D80E00E94981D0E94D41DFA
:10409000A196E6E00C94692EA0E0B0E0E2E5F0E243
:1040A0000C944B2ECAECD3E014E606E035E0F32E78
:1040B00044E0E42E53E0D52E62E0C62E82EE95E079
:1040C0000E94A82B892B09F49BC082EE95E00E94E8
:1040D000D52B282F809335044091340450E047308D
:1040E000510560F7FA01EE52FF4F0C94782E853B94
:1040F00029F781E080933404E1CF823609F07DC056
:10410000C0923404DBCF8093330480933204D09286
:104110003404D4CF9C0133273093310420933004EE
:1041200090913204982790933204E0923404C6CFE1
:10413000382F22274091300450913104242B352B05
:104140003093310420933004909132049827909357
:104150003204F09234042536310508F4AFCF61E023
:1041600070E08CEC0E94B71D81E00E94981D0E94B7
:10417000D41D43C020912E0430912F04F901E65341
:10418000FC4F808390913204982790933204C901A8
:10419000019690932F0480932E0420913004309147
:1041A00031048217930708F489CF0093340486CF33
:1041B0008091320482130BC060912E0470912F0401
:1041C0004AEC53E0809133040E94DB1D0DC062E095
:1041D00070E08BEC0E94B71D809133040E94981D03
:1041E00080916A050E94981DFE01812F11928A9587
:1041F000E9F710922F0410922E04109234045ECF2F
:10420000CDB7DEB7E8E00C94672E81E080936B05B4
:1042100080916B05882349F082EE95E00E94A82BDF
:10422000892BB1F30E944C20F3CF0895AAE2B0E0AD
:10423000ECE1F1E20C94492E0E949C286B017C0178
:1042400081E00E947E0A82EE95E00E94A82B892BD5
:1042500029F082EE95E00E94D52BF5CF5E9840982C
:1042600011E072E6B72EE9E2AE2E03E00E949C2830
:104270006C197D098E099F09693C710581059105BD
:10428000E0F11123D1F10E949C286B017C015D9A21
:10429000419A80ED97E00E94A807B982E6E7F5E031
:1042A000DE0112968A2D01900D928A95E1F76AE25D
:1042B000CE0101960E94DB0B5D98419880E090E072
:1042C0000E94A807009373050E94590B62E370E0F7
:1042D00080E090E00E94CB2880917305843061F4E7
:1042E000009373058FE70E9477090E948A0911E005
:1042F000823419F410E001C011E083E10E94C12969
:10430000892BA1F411E012C05E9A409A5D9A419AFD
:1043100082EE95E00E94D52B8D309105B9F06CF4BA
:104320000A97A1F05E9840985D98419882EE95E0DA
:104330000E94A82B892B41F799CF8332910579F000
:104340008234910579F70E940521ECCF62EB71E090
:1043500082EE95E00E94822A0E946E1DE3CF0E94A9
:10436000F715E0CF8F929F92AF92BF92CF92DF92DC
:10437000EF92FF921F93CF93DF9383E10E94C129B5
:10438000892B09F089C068EC70E080E090E00E9421
:10439000CB2880E090E00E94A8070E949C284B0157
:1043A0005C016B017C0180ECC80E82E1D81EE11C2F
:1043B000F11C0E949C286C157D058E059F0530F42C
:1043C00083E10E94C129892BA1F364C083E10E948B
:1043D000C129892B09F05EC080ED97E00E94A807F3
:1043E0000E949C286B017C01D0E0C1E088E4880E2B
:1043F00086E2981EA11CB11C11E083E10E94C12934
:10440000892B21F58C149D04AE04BF0430F480ED9B
:1044100097E00E94A807D1E0F0CF0E949C286C1979
:104420007D098E099F09693C71058105910528F375
:104430000E949C286B017C01C12719F080ED97E058
:1044400002C080E090E00E94A807D7CF80E090E013
:104450000E94A807DD23B9F08091D30590E0019672
:1044600065E070E00E94EC2D8093D3050E942B0D37
:104470000E94A9130E944A0D64EF71E080E090E071
:104480000E94CB2809C080E00E94DF060E94C21172
:104490000E94410D0E941621DF91CF911F91FF9044
:1044A000EF90DF90CF90BF90AF909F908F90089546
:1044B000CF92DF92EF92FF9280E00E94DA070E9493
:1044C000B10761E086E00E94552961E085E00E9425
:1044D000552961E08EE00E94552961E08FE00E943D
:1044E000552960E083E10E94552960E088E00E9440
:1044F000552961E088E00E948E290E949F0740E0D4
:1045000052EC61E070E082EE95E00E94F02C0E9497
:10451000A9130E944A0D0E948E138FEF8093AA0464
:104520000E94C60778940E949C286B017C018091B0
:10453000AA048F3F59F40E949C286C197D098E09AA
:104540009F09603D77408105910588F380ED97E0F4
:104550000E94A80761E083E10E948E295E9A409A3A
:1045600082EE95E00E94A82B892B29F082EE95E03F
:104570000E94D52BF5CF6DEF72E082EE95E00E94A0
:10458000632A84E893E00E94300C64E173E082EED9
:1045900095E00E94632A4AE050E069E070E082EE14
:1045A00095E00E94332B62E370E080E090E00E948F
:1045B000CB2882EE95E00E94A82B04970CF182EEA6
:1045C00095E00E94D52B82349105D1F482EE95E0DE
:1045D0000E94D52B8E34910599F482EE95E00E94CD
:1045E000D52B8434910561F482EE95E00E94D52BA1
:1045F000819731F480E090E00E94A8070E94162184
:1046000040917705509178056091790570917A0510
:10461000DB01CA010197A109B1090497A105B10500
:1046200068F44093A904433029F440EA56E861E075
:1046300070E004C040E052EC61E070E082EE95E092
:104640000E94F02C0E94B2215E98409880E090E099
:104650000E94A8070E948E131092C5048091BF0586
:1046600083FF11C080918B05882351F080919205C2
:10467000882331F080919905882311F087E001C0EB
:1046800085E08093C50480E00E947E0A8091C60484
:104690000E94B2090E94590B10923F0410923E04EE
:1046A00010923D04F12C8091D4058F15B0F062E397
:1046B00070E080E090E00E94CB2880ED97E00E94BF
:1046C000A80762E370E080E090E00E94CB2880E0E1
:1046D00090E00E94A807F394E6CF80919E0584FFA6
:1046E00008C0982F987181E0983109F080E00E940D
:1046F0007E118FE00E94DA07FF90EF90DF90CF905D
:104700000895EF92FF920F931F93CF93DF938C0145
:104710006EE770E082EE95E00E945906E801F12C08
:10472000F0E2EF2E8E0188818D57823048F46DE7DC
:1047300070E082EE95E00E94590688818E2588837C
:104740002196F801608182EE95E00E94022CF3949C
:10475000F9E0FF12E7CF6EE770E082EE95E00E948D
:104760005906CDB7DEB7E6E00C94692EA9E0B0E0BB
:10477000ECEBF3E20C94512E9091C70491110EC012
:104780009EEF99838A836B8350E0559547954C83C0
:104790002D83198618861F821E822EC04091CC045C
:1047A000842F90E0B4E095958795BA95E1F7242F92
:1047B0002F7030E08217930719F18DEF89831B82E8
:1047C000FE01349650E0842F90E0A4E09595879503
:1047D000AA95E1F7242F2F7030E08217930749F054
:1047E000DC01A353BB4F8C918193405F5F5F5630D8
:1047F00051F74093CC045A83CE0101960E94812345
:104800008091C70490E0019666E070E00E94EC2D74
:104810008093C7042996E2E00C946D2EA0E0B0E0EE
:10482000E4E1F4E20C944A2E6C016EE770E082EE53
:1048300095E00E9459068601E12CF12CC0E0D0E001
:1048400030E2B32EF801608183E8860F823078F47D
:104850006DE770E082EE95E00E945906F8016081F4
:104860006B2570E082EE95E00E94590604C082EE4E
:1048700095E00E94022CE114F10459F0F8018081C6
:104880009E01280F311DC901C92FDD27C80FD91F6F
:10489000DD273FEFE31AF30A89E0E816F10459F047
:1048A00028E0E216F10421F48C2F8095F601808730
:1048B0000F5F1F4FC7CFCDB7DEB7E9E00C94662E70
:1048C000A9E0B0E0E6E6F4E20C94512EE82F362F92
:1048D0008091C70490E0019664E270E00E94EC2DA4
:1048E0008093C70458E9598350E15A83813089F095
:1048F00048F08230B9F08330D9F48B8381EF8C8318
:104900003D8319C085E08B8381EF8C832F5F2D83DE
:1049100012C08B8381EF8C8384E6489FA001112411
:104920005D8309C084E08B8381EF8C83ED8303C0BA
:104930000E94BB1104C0CE0101960E940E2429964C
:10494000E2E00C946D2EA2E0B0E0E9EAF4E20C940F
:10495000462E182F762E2A8349830E94A8286B01A1
:104960007C018091DD048090C8049090C904A090DF
:10497000CA04B090CB042A8149818823C1F0D701B1
:10498000C60188199909AA09BB094C015D0191EE7C
:1049900089169EE29906A104B10420F1241708F4B7
:1049A000422F202F672D812F0E94602413C0D70132
:1049B000C60188199909AA09BB094C015D0191E357
:1049C000891695E79906A104B10460F0672D812F3F
:1049D0000E94B623C092C804D092C904E092CA04CF
:1049E000F092CB042296EDE00C94622EA2E2B0E0AD
:1049F000ECEFF4E20C94472E8CE00E9499098111AF
:104A00000FC06CE173E082EE95E00E94942A5E9AFA
:104A1000409A80E00E947E0A0E94590B5E9840985E
:104A200082EE95E00E94A82B892B01F182EE95E0A1
:104A30000E94D52B9091A904992319F00E94BC13D0
:104A4000EFCF40913E0450E09A012F5F3F4F2F710E
:104A5000332760913F0470E02617370709F3FA0106
:104A6000E75BFB4F808320933E04DACF8091730590
:104A7000843009F086C00E94A8286115710581055F
:104A8000910549F06093B7047093B8048093B9041A
:104A90009093BA040CC081E090E0A0E0B0E0809375
:104AA000B7049093B804A093B904B093BA0480916A
:104AB000AD049091AE0481609093AE048093AD04F8
:104AC00083E0809373058FE70E94770909E614E07D
:104AD0000E948A09F80181938F01F4E002371F07D1
:104AE000B9F72091720480916904982F922796FF5C
:104AF0003BC090E4922790937204982F9873983358
:104B0000F1F410E0212F30E080916904877090E08B
:104B1000821793074CF11F5F20919E05812F90E033
:104B2000FC01E759FB4F24FF04C080810E949D11C6
:104B3000E9CF608182EE95E00E94022CE3CF8F7373
:104B400099F480916A048093B60480916B048093F9
:104B5000B40480916C048093B30480916F0490E05E
:104B60009093AC048093AB0480913D04813019F4A0
:104B700082E080933D0480913D04833011F41092D3
:104B80003D040E94A8286B017C018091AF049091A4
:104B9000B004A091B104B091B2040097A105B10591
:104BA000C9F0A7019601281B390B4A0B5B0BDA01F0
:104BB000C901883B9B40A105B10560F00E94C8096E
:104BC0008093B5041092AF041092B0041092B10417
:104BD0001092B2048091BB049091BC04A091BD04DA
:104BE000B091BE0446015701881A990AAA0ABB0A65
:104BF00086E795E00E94F40786169706A806B90690
:104C000008F4A9C0C092BB04D092BC04E092BD04D9
:104C1000F092BE040E9457068091AA048830A0F04A
:104C20008091BF059091C005A091C105B091C205CA
:104C30005CE1B695A795979587955A95D1F7892BFD
:104C40008A2B8B2B09F0A2C18091AA048F5F8093DD
:104C5000AA048091B7049091B804A091B904B091CE
:104C6000BA040097A105B105F1F0C81AD90AEA0AF9
:104C7000FB0A86E795E00E94F4076C157D058E051A
:104C80009F0508F008C18091BF0584FD04C080ED38
:104C900097E00E94A8071092B7041092B8041092EF
:104CA000B9041092BA0490917204907C90937204AB
:104CB00050913E0480913F0420913D04581709F41F
:104CC00007C1223009F004C1905890937204E0911A
:104CD0009E05E770F0E0E658FC4F6081693008F00F
:104CE000DFC0615040E04613DDC080933F0487E39E
:104CF000840F90917204892B809372044093400436
:104D000083E080933D045D9A419A80918305909160
:104D1000C50491112CC10E94790A8091C6040E9499
:104D2000B209E0919E05E770F0E0E658FC4F608123
:104D300082E794E00E94940BE091C604EF5FE09359
:104D4000C604E83109F41FC1F0E0EA58FA4F87853C
:104D5000882309F418C10E94030C813069F5809101
:104D60009E05887149F18091AD049091AE04880F41
:104D7000991F9093AE048093AD0483E080937305F4
:104D80000E94590B0E94A8286093AF047093B0044E
:104D90008093B1049093B204672B682B692B61F464
:104DA00081E090E0A0E0B0E08093AF049093B00485
:104DB000A093B104B093B20480919E0584FF1FC0FC
:104DC0008091AD049091AE048E7F0E942A09182F25
:104DD0006091AB048091B6040E94B213482F612FFA
:104DE0008091B50449A30E94B2130091D405282FE5
:104DF00049A16091B3048091B4040E94A3245D98FA
:104E000041988091C3048130C1F018F08230B1F133
:104E1000CBC083E10E94C129892B09F0C5C081E084
:104E20008093C3040E949C286093BF047093C004C5
:104E30008093C1049093C204B7C083E10E94C1294A
:104E4000892B31F50E949C28C090BF04D090C004EB
:104E5000E090C104F090C2046C197D098E099F098D
:104E6000693E73408105910508F49EC082E08093FD
:104E7000C30480ED97E00E94A80796C083E10E94DA
:104E8000C129892B09F490C080E090E00E94A80716
:104E90001092C30489C080E090E00E94A80703CF6D
:104EA00068E020CF851709F420CF4F5F242F30E032
:104EB00090E0F901EE58FB4FDC01A75BBB4F7C9102
:104EC0007083F901E05CFB4F708301968F710BCF0B
:104ED0002430B1F42091400481E494E0A3E7B4E0ED
:104EE000FC013E2F381B321718F431913D93F9CF56
:104EF00087E3820F90917204892B8093720400CF14
:104F00008091C304823059F49160909372045E9A48
:104F1000409A8E010F5F1F4FF12CB80111C05E98AF
:104F2000409880913D04811103C081E080933D044D
:104F300080913D04833069F784E080933D04E9CF9C
:104F40008F2D69A37AA30E94B415F80181939193E0
:104F50008F01F39469A17AA1F0E1FF12F1CF809162
:104F60009E0543E754E087700E947908CCCE8823E1
:104F700009F4D1CE2091C40431E0320F3093C4043F
:104F80002913C9CE0DC01092C604E5CE8091AA04A3
:104F9000883011F45E9A409A89E08093AA04DBCEAF
:104FA0001092C4048150B7CEA296ECE00C94632E0C
:104FB0008230E8F4E82FF0E0EE0FFF1FEB52FA4FDB
:104FC00071836083813041F0809169008C7F842BF4
:104FD00080936900E89A089580916900440F551FF5
:104FE000440F551F837F842B80936900E99A0895AD
:104FF0001F920F920FB60F9211242F933F934F934E
:105000005F936F937F938F939F93AF93BF93EF9330
:10501000FF938091D5059091D605892B29F0E091D9
:10502000D505F091D6050995FF91EF91BF91AF910C
:105030009F918F917F916F915F914F913F912F91B0
:105040000F900FBE0F901F9018951F920F920FB6E2
:105050000F9211242F933F934F935F936F937F93FE
:105060008F939F93AF93BF93EF93FF938091D70557
:105070009091D805892B29F0E091D705F091D805BA
:105080000995FF91EF91BF91AF919F918F917F9182
:105090006F915F914F913F912F910F900FBE0F90A5
:1050A0001F9018951F920F920FB60F9211242F93F5
:1050B0003F938F939F93AF93BF938091DA05909125
:1050C000DB05A091DC05B091DD053091D90523E029
:1050D000230F2D3720F40196A11DB11D05C026E830
:1050E000230F0296A11DB11D2093D9058093DA05E7
:1050F0009093DB05A093DC05B093DD058091DE0580
:105100009091DF05A091E005B091E1050196A11D08
:10511000B11D8093DE059093DF05A093E005B09369
:10512000E105BF91AF919F918F913F912F910F908A
:105130000FBE0F901F9018952FB7F8946091DA0565
:105140007091DB058091DC059091DD052FBF0895FE
:105150003FB7F8948091DE059091DF05A091E005BE
:10516000B091E10526B5A89B05C02F3F19F0019627
:10517000A11DB11D3FBF6627782F892F9A2F620F7F
:10518000711D811D911D42E0660F771F881F991FB9
:105190004A95D1F70895CF92DF92EF92FF92CF9385
:1051A000DF936B017C010E94A828EB01C114D1049C
:1051B000E104F10479F00E94A8286C1B7D0B683E85
:1051C0007340A0F381E0C81AD108E108F108C85182
:1051D000DC4FECCFDF91CF91FF90EF90DF90CF903D
:1051E0000895789484B5826084BD84B5816084BD5F
:1051F00085B5826085BD85B5816085BDEEE6F0E050
:10520000808181608083E1E8F0E0108280818260AB
:105210008083808181608083E0E8F0E0808181602C
:105220008083E1EBF0E0808184608083E0EBF0E05C
:10523000808181608083EAE7F0E080818460808300
:1052400080818260808380818160808380818068AA
:1052500080831092C1000895833081F028F481305A
:1052600099F08230A1F008958630A9F08730B9F026
:105270008430D1F4809180008F7D03C080918000C4
:105280008F7780938000089584B58F7702C084B5AE
:105290008F7D84BD08958091B0008F7703C0809189
:1052A000B0008F7D8093B0000895CF93DF9390E09E
:1052B000FC01ED50F44F2491FC01E95FF34F849120
:1052C000882349F190E0880F991FFC01E15DF34FBD
:1052D000A591B4918B5D934FFC01C591D4919FB77B
:1052E000611108C0F8948C91209582238C93888159
:1052F00082230AC0623051F4F8948C91322F309599
:1053000083238C938881822B888304C0F8948C91AA
:10531000822B8C939FBFDF91CF910895A1E0B0E0E5
:10532000E4E9F9E20C944F2E282F30E0F901E15224
:10533000F44F8491F901ED50F44F1491F901E95FB4
:10534000F34F04910023C9F0882321F069830E9460
:105350002C296981E02FF0E0EE0FFF1FEB5DF34F8A
:10536000A591B4919FB7F8948C91611103C01095E9
:10537000812301C0812B8C939FBF2196E4E00C9484
:105380006B2ECF93DF93282F30E0F901E152F44FD9
:105390008491F901ED50F44FD491F901E95FF34F95
:1053A000C491CC2391F081110E942C29EC2FF0E0C4
:1053B000EE0FFF1FE55EF34FA591B4912C912D23C5
:1053C00081E090E021F480E002C080E090E0DF9195
:1053D000CF9108958E3008F08E50877020919D01F6
:1053E00090E4299F90011124822B80937C0080916E
:1053F0007A00806480937A0080917A0086FDFCCFE9
:10540000809178002091790090E0922B0895A0E09F
:10541000B0E0EDE0FAE20C944B2E6C017A01EB0166
:10542000E60EF71E00E010E0CE15DF0561F0699191
:10543000D601ED91FC910190F081E02DC601099516
:10544000080F191FF1CFC801CDB7DEB7E8E00C9403
:10545000672E6115710589F0DB010D900020E9F7D9
:10546000AD0141505109461B570BDC01ED91FC91F8
:105470000280F381E02D0995089580E090E0089581
:10548000EF92FF920F931F93CF93DF938C01FB0159
:10549000C0E0D0E064917F018FEFE81AF80A66233C
:1054A00061F0D801ED91FC910190F081E02DC801EF
:1054B0000995C80FD91FF701EDCFCE01CDB7DEB7E3
:1054C000E6E00C94692E0E94292A0895DC01ED91F2
:1054D000FC910190F081E02D099508950F931F93A1
:1054E000CF93DF93EC016DE00E94662A8C016AE0A5
:1054F000CE010E94662A800F911FDF91CF911F91EC
:105500000F9108950F931F93CF93DF93EC010E94A7
:10551000402A8C01CE010E946E2A800F911FDF91DC
:10552000CF911F910F9108950F931F93CF93DF9306
:10553000EC010E94292A8C01CE010E946E2A800F64
:10554000911FDF91CF911F910F9108950F931F939A
:10555000CF93DF93EC010E94662A8C01CE010E945A
:105560006E2A800F911FDF91CF911F910F910895A7
:10557000A1E2B0E0EEEBFAE20C94472E7C01C42EDF
:10558000E52FCB01D22E19A221E02D1510F02AE033
:10559000D22E8E010F5D1F4F8D2C912CA12CB12C82
:1055A0006C2D7E2FA50194010E94002E8C2DD29E81
:1055B00080191124015011098A3010F4805D01C056
:1055C000895CF8018083211531054105510521F0E1
:1055D000C22EE32FCA01E4CFB801C7010E94292AD5
:1055E000A196ECE00C94632EA0E0B0E0EAEFFAE2C2
:1055F0000C944B2EEC016A017B012115310541F41D
:10560000E881F9810190F081E02D642F09951DC09A
:105610002A303105A9F477FF12C06DE20E94662A94
:105620008C0144275527BA014C195D096E097F0981
:105630002AE0CE010E94B82A800F911F06C02AE0FE
:10564000B701A601CE010E94B82ACDB7DEB7E8E0C7
:105650000C94672E9A01AB01662757FD6095762F53
:105660000E94F42A08950F931F93CF93DF93EC01C8
:105670009A01AB01662757FD6095762F0E94F42AA8
:105680008C01CE010E946E2A800F911FDF91CF9175
:105690001F910F9108952115310549F4DC01ED9119
:1056A000FC910190F081E02D642F099508950E94EE
:1056B000B82A08959A01462F50E060E070E00E94F9
:1056C0004B2B08959A01AB0160E070E00E944B2BD8
:1056D00008950F931F93CF93DF93EC010E944B2B00
:1056E0008C01CE010E946E2A800F911FDF91CF9115
:1056F0001F910F9108950F931F93CF93DF93EC01A8
:105700009A01AB0160E070E00E944B2B8C01CE014E
:105710000E946E2A800F911FDF91CF911F910F91F0
:1057200008950F931F93CF93DF93EC019A01462FB7
:1057300050E060E070E00E944B2B8C01CE010E9493
:105740006E2A800F911FDF91CF911F910F910895C5
:10575000FC0124853585F901E05CFF4F8081918152
:10576000F901EE5BFF4F20813181821B930B8F7318
:1057700099270895FC0184859585FC01E05CFF4F25
:1057800040815181FC01EE5BFF4F20813181421746
:10579000530741F00190F081E02DE80FF91F80815F
:1057A00090E008958FEF9FEF0895FC018485958523
:1057B000FC01E05CFF4F40815181FC01EE5BFF4F3B
:1057C000208131814217530779F0A081B181A80F60
:1057D000B91F8C91208131812F5F3F4F2F73332769
:1057E0003183208390E008958FEF9FEF0895FC01AF
:1057F00081A1882329F0A489B5898C9186FFFBCFEC
:1058000011A20895CF93DF93FC0126853785D90136
:10581000A05CBF4F8D919C91119701968F73992732
:10582000E901CE5BDF4F4881598184179507D9F391
:105830000D90BC91A02DA20FB31F6C93A685B785C8
:10584000A05CBF4F11969C938E93A689B7892C912B
:1058500081E090E0078C02C0880F991F0A94E2F75C
:10586000282B2C9381E081A30488F589E02D808189
:105870008064808381E090E0DF91CF910895089566
:105880001F920F920FB60F9211242F933F934F93B5
:105890008F939F93EF93FF938091C00082FD1CC074
:1058A0004091C600809188069091890601968F7379
:1058B000992720918A0630918B068217930771F001
:1058C000E0918806F0918906E85BF94F4083909358
:1058D00089068093880602C08091C600FF91EF91EF
:1058E0009F918F914F913F912F910F900FBE0F90ED
:1058F0001F90189582EE95E00E94A82B892B11F03D
:105900000E943F2C08951F920F920FB60F92112400
:105910002F933F938F939F93EF93FF932091440690
:105920003091450680914606909147062817390721
:1059300031F48091C1008F7D8093C10014C0E0914B
:105940004606F0914706EC5FF94F208180914606AC
:105950009091470601968F739927909347068093FD
:1059600046062093C600FF91EF919F918F913F9142
:105970002F910F900FBE0F901F901895A0E0B0E0F0
:10598000E4ECFCE20C94472EFC011382128288EEB8
:1059900093E0A0E0B0E084839583A683B7838CEB8B
:1059A00093E0918380837587648757874687318B1F
:1059B000208B138B028BF58AE48AD78AC68AB18E34
:1059C000A08E938E828E8F85848F8889858F89891A
:1059D000868F8A89878F8B8980A3ECE00C94632E55
:1059E000CF92DF92EF92FF92CF93DF93EC016A01A7
:1059F0007B01411581EE580761057105F9F0EC89CD
:105A0000FD8981E090E008A002C0880F991F0A94E8
:105A1000E2F7808360E079E08DE390E0A7019601F2
:105A20000E94002E21503109410951095695479590
:105A300037952795211580E1380798F0EC89FD8985
:105A4000108260E874E88EE190E0A70196010E9460
:105A5000002E215031094109510956954795379536
:105A60002795E889F9893083EA89FB89208319A27F
:105A7000EE89FF89408181E090E09C010C8C02C09E
:105A8000220F331F0A94E2F7422B4083EE89FF89ED
:105A900040819C010D8C02C0220F331F0A94E2F753
:105AA000422B4083EE89FF8940819C010E8C02C00D
:105AB000220F331F0A94E2F7422B4083EE89FF89BD
:105AC00020810F8C02C0880F991F0A94E2F78095FD
:105AD00082238083DF91CF91FF90EF90DF90CF9072
:105AE00008958F929F92AF92BF92CF92DF92EF92E2
:105AF000FF920F931F9381E08F9385E08F9387E050
:105B00008F9383E08F9384E08F93E6EC8E2E912C1D
:105B1000F2ECAF2EB12CA1ECCA2ED12CB0ECEB2EB6
:105B2000F12C04EC10E025EC30E044E056E068E4B1
:105B300076E082EE95E00E94BE2C0F900F900F90C1
:105B40000F900F901F910F91FF90EF90DF90CF90EB
:105B5000BF90AF909F908F9008950E94F1280E946F
:105B60005822CAE7DCE20E94F6242097E1F30E9463
:105B70007A2CF9CFA29FB001B39FC001A39F700DF3
:105B8000811D1124911DB29F700D811D1124911D45
:105B900008950E94BA2DA59F900DB49F900DA49FCB
:105BA000800D911D11240895B7FF0C94C92D0E94FA
:105BB000C92D821B930B0895DB018F939F930E9445
:105BC000C92DBF91AF91A29F800D911DA39F900DF4
:105BD000B29F900D1124089597FB072E16F40094A0
:105BE00007D077FD09D00E947E2E07FC05D03EF439
:105BF000909581959F4F0895709561957F4F089579
:105C0000A1E21A2EAA1BBB1BFD010DC0AA1FBB1FC0
:105C1000EE1FFF1FA217B307E407F50720F0A21B32
:105C2000B30BE40BF50B661F771F881F991F1A949F
:105C300069F760957095809590959B01AC01BD01C9
:105C4000CF010895052E97FB1EF400940E94392E73
:105C500057FD07D00E94002E07FC03D04EF40C9491
:105C6000392E50954095309521953F4F4F4F5F4FBE
:105C7000089590958095709561957F4F8F4F9F4FB8
:105C800008952F923F924F925F926F927F928F92E0
:105C90009F92AF92BF92CF92DF92EF92FF920F93BB
:105CA0001F93CF93DF93CDB7DEB7CA1BDB0B0FB6C5
:105CB000F894DEBF0FBECDBF09942A883988488882
:105CC0005F846E847D848C849B84AA84B984C88418
:105CD000DF80EE80FD800C811B81AA81B981CE0F0F
:105CE000D11D0FB6F894DEBF0FBECDBFED010895F4
:105CF000EE0FFF1F0590F491E02D0994AA1BBB1B2A
:105D000051E107C0AA1FBB1FA617B70710F0A61BBB
:105D1000B70B881F991F5A95A9F780959095BC01DC
:105D2000CD0108958F929F92AF92BF92CF92DF9252
:105D3000EF92FF92CF93DF93EC01688179818A81A2
:105D40009B81611571058105910521F464E279ED6E
:105D50008BE597E02DE133EF41E050E00E94222EE9
:105D600049015A019B01AC01A7EAB1E40E94C92D87
:105D70006B017C01ACEEB4EFA50194010E94D72D1C
:105D8000C60ED71EE81EF91EF7FE06C081E0C81A2F
:105D9000D108E10880E8F80AC882D982EA82FB8249
:105DA000C701B6019F77DF91CF91FF90EF90DF9011
:105DB000CF90BF90AF909F908F9008950E94922EA9
:105DC000089586E091E00E94922E08956093060166
:105DD00070930701809308019093090108952F9211
:105DE0003F925F926F927F928F929F92AF92BF92FB
:105DF000CF92DF92EF92FF920F931F93CF93DF9397
:105E00008B01EA016115710521F0DB018C9311967C
:105E10009C93209739F09E0122503109233231059D
:105E200008F0D8C07C016701BFEFCB1ADB0A56012E
:105E3000F7016080862D90E00E942130892B11F0BF
:105E40007601F1CFFDE26F120AC0570182E0A80E81
:105E5000B11CD70111966C90772473940BC0BBE2F0
:105E60006B1207C05701E2E0AE0EB11CD7011196CC
:105E70006C90712CCE018F7E892B89F4B0E36B126C
:105E800037C0F50180818F7D8835D1F46180F2E0E3
:105E9000AF0EB11C872D8260782EC0E1D0E0CA30F1
:105EA000D10551F1C031D10521F0C830D10599F4A7
:105EB00009C0CC24CA94DC2CEC2CAFE0FA2E22C012
:105EC000209769F7C8E0D0E0CC24CA94DC2CEC2CF5
:105ED000FFE1FF2E17C06FEF7FEFCB019E0144273C
:105EE00037FD4095542F0E94002E69017A010AC0A7
:105EF0002097A9F6CAE0D0E0E9E9CE2EDC2CEC2C04
:105F0000E9E1FE2EF50160E020E030E0A9014E015C
:105F1000AA2497FCA094BA2C1F0170ED572E560CA2
:105F2000A9E0A51570F48FEB860D8A3118F499EC71
:105F3000592E06C08FE9860D8A3148F589EA582E18
:105F4000560C852D90E08C179D070CF56F3FD9F00E
:105F5000C216D306E406F50698F0C501B4010E9406
:105F6000DC2D9B01AC01852D90E0A0E0B0E0280F76
:105F7000391F4A1F5B1F281739074A075B0710F4B0
:105F80006FEF01C061E03196D1016C90C5CF011572
:105F9000110551F0662311F0319703C071FE04C062
:105FA0003297D801ED93FC9370FE07C05095409551
:105FB000309521953F4F4F4F5F4F67FF10C082E2F2
:105FC00090E090938D0680938C066FEF7FEF8FEFBC
:105FD0009FEF07C060E070E080E090E002C0B90190
:105FE000CA01DF91CF911F910F91FF90EF90DF9049
:105FF000CF90BF90AF909F908F907F906F905F9069
:106000003F902F900895FC0188279927E8942191CB
:106010002032E9F3293010F02E30C8F32B3241F052
:106020002D3239F4689404C00E945530820F911DBE
:10603000219120532A30C0F31EF4909581959F4FF3
:106040000895911150C0803219F089508550D0F7D1
:10605000089548EC53E00E942E300895FA01A19172
:10606000B081009719F41097E1F0CD01DC01CD016A
:106070000D90002011F4C00113C0FB0121912223D7
:1060800019F02015D9F7F3CFFB012191201519F450
:106090001E92119606C02223C1F70D900020A1F791
:1060A000D001FA01A193B08308957AE0979F902DD3
:1060B000879F802D910D11240895F999FECF92BDEF
:1060C00081BDF89A992780B50895262FF999FECFBA
:1060D0001FBA92BD81BD20BD0FB6F894FA9AF99A05
:1060E0000FBE01960895992788270895F894FFCF49
:1060F00000008E06200001000000FF0002000200E8
:10610000020002000200020002000200020002007F
:1061100002000200020002000200028025000005C9
:10612000400AA1204EA50020244EA52C2330C012E9
:1061300000001A400AA1204EA5001B1E27522C2346
:10614000308025000005400AA1204EA50020244EE5
:10615000A52C2330004B000006400AD0009D4900CA
:106160007B289D492C233000E1000005400A4501B1
:10617000D7DC03B81E0EBF00232E48E801008A407A
:106180000A6001555502AD1E20000023C801545875
:106190002074696D656F75742100596573004E6FC9
:1061A000002C00386368004E2F41002C205B005DFE
:1061B0002028002900486F70206368616E6E656C4E
:1061C000200020402000456E746572696E67206172
:1061D00064617074697665206368616E6E656C20B9
:1061E00073656C656374696F6E2C207069636B698D
:1061F0006E673A007363616E6E6572206D6F6465E1
:10620000004E4F5420454E41424C45440053656E6C
:1062100064696E672073657474696E677320746F48
:106220002052580A00526573657474696E67207352
:10623000657474696E6773206F6E2052580A00414E
:10624000626F727465642065646974730A00696EB4
:1062500076616C69642073656C656374696F6E0048
:106260000D0A496E76616C696420696E70757420E0
:106270002D2064697363617264656421070053654E
:106280007474696E677320736176656420746F201F
:10629000454550524F4D0A005265766572746564EB
:1062A0002073657474696E67732066726F6D204524
:1062B0004550524F4D0A004C6F6164656420666121
:1062C00063746F72792064656661756C74730A001B
:1062D0004B657920616E64206368616E6E656C73D6
:1062E0002072616E646F6D697A65640A004F706533
:1062F0006E4C52536E6720545820737461727469E7
:106300006E672000206F6E20485720006D6F647507
:106310006C65206C6F636B65643F00342B34003810
:1063200000382B340031320031322B34003136004A
:1063300050504D0052535349005344410053434C75
:1063400000525844005458440041494E004C4245C4
:1063500045500053504B54524D0053425553005337
:10636000554D44004C4C494E440000070B0C101195
:106370001500B7012B032F033103350338033D0309
:10638000B7014003440349034D0351035503590327
:106390005D0363036A036F0374038D028D028D0234
:1063A0008D02160A1322312900000000022C072A50
:0863B000A82BD52BBA2BF72B0B
:107E00000F92CDB7DEB7112484B714BE81FFF1D035
:107E100082E08093C00088E18093C10086E0809377
:107E2000C20080E18093C4008EE0CDD088249924E4
:107E3000CC24C394F5E0DF2EE1E1EE2E73E0F72EC3
:107E4000B6D0082F813479F4B2D08983C2D0898129
:107E5000823811F481E005C0813811F485E001C059
:107E600083E09ED09AC0823411F484E103C085344B
:107E700019F485E0B6D091C0853561F498D0082F0B
:107E800010E095D090E0982E8824802A912A880CC2
:107E9000991C82C0863521F484E0A3D080E0E1CF34
:107EA000843609F04CC083D082D0A82E80D0B82E62
:107EB00000E011E07CD0F80181938F01AE16D1F77C
:107EC00088D0FB2DF53489F4E0E0F1E00BC0F9999E
:107ED000FECF92BC81BC0894811C911C819180BD15
:107EE000FA9AF99AEA1598F358C08B2D863409F05E
:107EF00054C0F401F7BEE89507B600FCFDCFF401CD
:107F0000A0E0B1E02C9130E011968C91119790E0B7
:107F1000982F8827822B932B12960C01C7BEE895C9
:107F20001124329681E0A038B80761F7F401D7BE7A
:107F3000E89507B600FCFDCFE7BEE8952EC0843774
:107F4000F1F435D034D0182F32D0B82E42D0FB2DDA
:107F5000F63421F4F40105914F010CC0FB2DF534EA
:107F600049F4F999FECF92BC81BC0894811C911C04
:107F7000F89A00B5802F14D0115049F70EC08537FC
:107F800039F427D08EE10CD085E90AD08FE069CF93
:107F9000813511F488E017D01CD080E101D050CF9A
:107FA0009091C00095FFFCCF8093C600089580910A
:107FB000C00087FFFCCF8091C00084FD01C0A89560
:107FC0008091C6000895E0E6F0E098E19083808318
:107FD0000895EDDF803219F088E0F5DFFFCF84E10E
:107FE000DFCF1F93182FE3DF1150E9F7F2DF1F9166
:0E7FF0000895282E80E0E7DFEE27FF27099492
:027FFE0001057B
:0400000300007E007B
:00000001FF
